:03F0000002F00813
:03F0610002F003B7
:05F0030012F06480FE24
:02F064007A0030
:03F06600BA4000AD
:0DF06900500B8A827583FE74FFF00A80F060
:05F07600C2A875E104D1
:0BF07B0090DF3BE0FABA01F875E102FB
:0DF0860090DF3BE0FABA0DF890DF02E09059
:05F09300FE00F07A010F
:0AF0980090DF02E0FBC3EA9B501377
:05F0A20010890280FB53
:0EF0A7008A030A8B827583FEE5D9FBF080E3B5
:05F0B50075E104A52235
:06F03700E478FFF6D8FDAD
:08F015007900E94400601B7A58
:05F01D000090F0BE7838
:03F02200007593E3
:0AF0250000E493F2A308B80002050E
:08F02F0093D9F4DAF27593FFA6
:08F03D007800E84400600A7944
:03F04500007593C0
:06F0480000E4F309D8FC0E
:08F04E007800E84400600C7931
:0BF0560000900000E4F0A3D8FCD9FA01
:03F0080075810708
:0AF00B0012F0BAE582600302F00380
:04F0BA007582002239
:00000001FF
